:020000040000FA
:10000000AE2A3E3477347F34773477343F347734D4
:100010003F3477343F343E347734073477343E34DA
:100020003F347734773477343F347F3407343F3488
:1000300007347F347F3407343F34073407347E3449
:100040000734773477347E34773477347F347734B9
:1000500077341C341C341C341C341C34383438348D
:10006000383438341E3477343F341F343F347734D7
:1000700007340734073407347F34633477347F34EC
:100080007F347734733477347F34773467343E3455
:100090007734773477343E343F3477343F34073421
:1000A00007343E34773477343F346E343F3477341A
:1000B0003F34773477347E3407343E3470343F3401
:1000C0007F341C341C341C341C347734773477343C
:1000D00077343E34773477343E343E341C347734CE
:1000E0007F347F347734633477343E341C343E3489
:1000F000773477343E341C341C341C347F34383429
:100100001C340E347F3400340034003400340034A6
:100110001C349901770883169B001C141A0883125B
:10012000F70A9900760883169B001C141A0883129C
:10013000F60A9900750883169B001C141A0883128E
:10014000F50A9900740883169B001C141A08831280
:10015000F40A9900730883169B001C141A08831272
:10016000F30A9900E1285025F000E4204C3057268E
:1001700099011812E420892099017808A02199009A
:100180007908A02199007A08A021990070083639D1
:10019000031D0130F807F907FA07181650257008F3
:1001A000F007031DB62808004408C5070318C60A4F
:1001B00046080F3995000800CA01C901C401803002
:1001C000CB000000000000000800F600F700F60E6B
:1001D000F030F605F7050310F60CF70C0800A00741
:1001E000A107A207A307A407A50708006108050641
:1001F0001C3AE1061039610508000000AC2EF82E0B
:100200004230F40018305E2D1030F4000830792DA3
:100210005430F4002A305E2D0030F4000030792D87
:100220004430F40004305E2D3830F4001C30792D59
:100230000030F4000030792D1030F4000830792DB2
:100240008830F40002305E2D3830F4001C30792DF7
:100250000030F4000030792D1030F4000830792D92
:100260009030F40002305E2D1030F40008305E2D26
:100270001030F40008305E2D0030F4000030962D70
:10028000FC30F4003F30AB2DF930F4009F30962D58
:100290009130F4001F305E2D0230F4004030962D76
:1002A0009E30F4007F30AB2DFF30F400FF30962DF0
:1002B000FD30F4007F305E2D3130F4008C30962D0F
:1002C000FE30F4007930AB2DFD30F400BF30962DB8
:1002D000FE30F400BF305E2DE130F4008730962D03
:1002E000FC30F4003F30AB2DF830F4001F30962D79
:1002F000F830F40089305E2D0230F4004030962D45
:100300001030F40008305E2D1030F40008305E2DFF
:100310002030F40004305E2D7830F4001E305E2D65
:100320000830F40010305E2D0830F40010305E2DDF
:100330000430F40020305E2D1E30F40078305E2D45
:1003400082002626E5252126D930D000DC205A0857
:10035000031D512A683084006822FB006822FC00DB
:10036000203084000630F00060308000053E840AB2
:10037000F00BB5297522EF207522FF30EF207F08A2
:10038000031DD3292508FD00250A83168F229B0310
:100390007C02031DCD2990227B02831205300319B4
:1003A000FF00031CFF007F08FE3E0318E1297B08C5
:1003B0007F187C085A22FF0A0130FE000509E1007F
:1003C000512AF620031D0E2A7F08053A03190F2A29
:1003D00061080C390319012AE20A62080F39031D6A
:1003E000032A0C30621AE2007E08053EE11DF63E4B
:1003F000FC3A03197F30743A03198930883AFE00B9
:10040000032AFF30E2007D087F0783168F227E06D5
:1004100003190F2A7E085A228312512AFF0A8312D7
:100420002030E7000630F2003030F3006708840027
:1004300083168E22E5207708F5007608F4009B0AE3
:100440009022E5209C22F8009C22F9009C22FA00D0
:100450008312B320F30A5025F30B2B2AE70AF20B81
:10046000162A7F08063A031D512A0330E600FF01D1
:100470000130EF0033252C30DF000230DB00E301D8
:10048000D83084001830F0007E30A3225025203070
:1004900084001330F0008317F730A3228313A822BF
:1004A000E40150255008031D512A2626E525133066
:1004B0006326262D83169A007D087F079B001C1556
:1004C00055309D00AA309D009C141C118312080019
:1004D000000E8739F000840A00087839F004840A95
:1004E000700870070318013E0800782277227822EE
:1004F000203084007E227C2250257E2283168E228C
:10050000F000840A8E227002000884030006031C97
:100510008006840A031C80068312013400089B00B5
:100520001C141A0808009B0A7D087F071B06031D80
:10053000902AF11D902A83349322FF3E7C3E0318BB
:100540008434853E08008000840AF00BA32A08004A
:10055000E801E901EA01EB01DA0108008501860101
:1005600007309F008316FC30850016308600B030BF
:1005700098000F3092009901831290309800053056
:1005800092000C30970090018A0186160530FF001A
:10059000EC00E601FF30EE00A822E5257530572675
:1005A0000B2605260B2605260B26F725FF25F72506
:1005B000FF25F7250B2605260B2605260B26E52508
:1005C000F82264000000E525F52505260B26052602
:1005D0000B260526FF25F725FF25F725FF250526F0
:1005E0000B2605260B2605260B26E525F822CD2A07
:1005F000F10A0E3063262D30D0001D30D200E525E3
:10060000212666080319F02B2030F00045275025DD
:10061000452750254527502548256418562B03109B
:10062000EC0C8E300318EC066C0807394326831354
:100630004330840000087605031D222B8403041B2D
:100640001A2B452B040E0B3E5507E7007508F507DE
:10065000F50704080339013E530256080318F5074D
:100660005408F507F50E750CF50C6C0E0739043EB1
:10067000F50783172C3084000008103E031C452B1F
:1006800067088000840A75088000F620EE1B0319B5
:10069000562B8317303084005B080319562BCF305C
:1006A0008000840A5F08083E8000DB03502548254F
:1006B0002030F000E700A030E000F40114275025BE
:1006C000132750251327502513275025132760087B
:1006D0008400FF3080005025640840044104420437
:1006E0004304F00070187F2B0330D407C00CC10CFA
:1006F000C20CC30CD70B842BE60A3325842B57037B
:10070000432670050319D7034308031D952BEF30CB
:100710005507031C952BF030D5074208C30041084C
:10072000C2004008C100C001ED036418F02B023084
:10073000851DDF075F08293ED7300318DF0003144B
:10074000FE30051DDF07031CDF015F084326DD00C7
:100750005D03DE005F0CDC00DC0C5C0C1F39203E0E
:10076000DC00D903031DC92B5808D900530A0339EB
:10077000D300031DC92B5608D40754257003D61F78
:100780007208031DC92BFE30D6060430D507D51BD1
:10079000D5025308403E84005307603CC400000863
:1007A0000319C4015908FD3E0318C4014A0803197E
:1007B000C7010319C801031DCA0363080319EB2B02
:1007C0007118E30A6308DF3A0319E30163080F397C
:1007D0008038C400F02B6C0871041F390319E30A38
:1007E0005025C030CB06EE1FEE0BE60AE6035A0892
:1007F0000319092CDA0368308400800A0008B73E28
:10080000031C092CF93E003003198000840A041DE2
:10081000FD2B0830D100F3016808F4006908F500E9
:100820006A08F6006B08F7005025500B142C26269A
:10083000E525073057268A011730F000660AE700E1
:100840005108FC3E7F309901181203180830E70365
:100850000319003000009900F00B272C2F2C00000A
:100860008920181604305726D10B182C0000E525D6
:10087000212666080319A1293C30840080018403E5
:10088000841A3E2CA030E000F7010A145508FA0043
:10089000783CFB005608D4076D0E3039F600F60799
:1008A0007608F6070430F4002626E5254E26582C57
:1008B0008506E420E22085065D2C5526E5254E269A
:1008C00000008506632C2F25652C85060000552623
:1008D000E5254E268506E120E12085065526E525FD
:1008E0004E262F252F255526E52507306326D725AB
:1008F0000A30572634260000FA0B772C0000D72543
:10090000E12077085306003003195608D40277080F
:10091000403E84000008F8000C30F900E420342642
:10092000F4030319A22C0000D7257719C92C6030D5
:100930005418103EFC00003054183030FD00E12007
:10094000E3208F2CD72554257808F300203084002D
:10095000760E76197D06F6197C0882007208031956
:10096000B82C00089900840AB52CF20BB12CB82CD5
:100970001816F60A0430FC07F90BA22C0000D72544
:10098000F70A3430F6070330F400812CD725C82C41
:100990000000FB037B08003CFB1F0030F900FB1B41
:1009A000FB01FB0AE120E32034260000FB0BC62CF0
:1009B0000000D725203084000430F40079080E3977
:1009C000F5000310750CF507D830F5077908F0002D
:1009D000F00C700C7906FE38E42099011812990188
:1009E0008A010000A021E4201816F62CF90A791ECD
:1009F000D92CF901D7250A3057263426F90AF91DD2
:100A0000FA2CF901D7255C0A84005D08EE188004F1
:100A1000053057263426F90A791D022DF901D7250C
:100A20005C0884005E09EE188004840AFF30EE182A
:100A30008000840A5E08EE188004E420E120342659
:100A4000F90A791D0F2DF901E120E120E525123089
:100A50006326D20B262D0000E5251330632E850674
:100A6000312D85060800FF30C000C100C200C30060
:100A70000130D400D600D3000830D7006F08D5006D
:100A80000830EF1FEF07ED012030D800D900080033
:100A900049254A254B2520308400FD265025FD267A
:100AA000D0032626E525212E5408F0005708E7003C
:100AB0006707670770071D3CF2000800F500990101
:100AC000C125F30C031C722D840A74089900840A52
:100AD000E320750899000008840AE4209900E70BD8
:100AE000612DAE2C00089900840A0008840A782D34
:100AF0006A2DF5009901C125F30C031C922D840A7F
:100B000074089900840A00000514862D05107508E4
:100B10009900000805148C2D0510840A9900E70B34
:100B20007C2DAE2C00089900C8258E2DF50099016A
:100B3000C125F30C031CA72D840A74089900840AAC
:100B40000514D02505109900E70B992DAE2C00084F
:100B50009900C825A32DF5009901C125F30C031CAC
:100B6000BC2D840A74089900840A8514D025851048
:100B70009900E70BAE2DAE2C00089900C825B82DC2
:100B8000000018120008840A9900F00BC02D08001C
:100B9000C92D840A0008840A99000008840A080004
:100BA000D12D750899000008840A0000080060082B
:100BB0008400800B112E840A0008F000840A0008CB
:100BC0008400700880060330E0070610D42000007F
:100BD0000310C80CC70C49080318C7060318C80639
:100BE00047084B058606061408001330632E0610CE
:100BF000D42013265F30572606140730572E0610D0
:100C00007930572606140730572E0610D4200614C4
:100C100013267430572E0610E420E120061483308A
:100C2000572EE120E52D0310C80CC70C4908031806
:100C3000C7060318C80647084B0586060800F930A2
:100C4000222EE9308E008F01101401340F08031991
:100C5000262E0E182B2E8E182D2E0E182F2E0E0827
:100C6000031D2F2E101008001D30F00020308400CE
:100C7000990118120008840A3D2E9900F00B3A2EB3
:100C8000E12018160800F5000130F5180430F600D0
:100C90007518F6077519F60E760808006308103EF9
:100CA00057266308031D013008006308DE3CFC3E44
:100CB0000318572E023E031C5F2EFE3E5F2E013EA0
:100CC000031CF134F1345726572E700CF00600083F
:100CD0009900840A0008840A99000008E700840A41
:100CE0000008F200840A0008F300840A67089900EB
:100CF000033070188506720899000330F0188506D5
:100D00007019850600007308990003300000F0197F
:100D10008506701A85060008990003300000F01A55
:100D20008506701B8506840A00089900040AE700FE
:100D3000750884000008F000670884000008990026
:100D4000840AF50AF40B652E00089900840A040849
:100D5000C33E031DA42E080000089900AF2E00001A
:100D6000932E700CF00600089900840A0008840A8B
:100D700099000008E700840A0008F200840A0008CD
:100D8000F300840A6708990003307018850672081A
:100D9000990003300000F018850670198506F019D7
:100DA0008506730899000330701A85060000000854
:100DB00099000330F01A85060000701B8506840A2E
:100DC00000089900040AE700750884000008F00094
:100DD0006708840000089900840AF50AF40BB12E14
:100DE00000089900840A0408C33E031DF02E080081
:100DF00000089900FB2E0000DF2E0830F200831758
:100E00000008840A840A721C000200088403840318
:100E10000006031C8006840A840A031C80068403DF
:100E2000F20B002F08001427152783177008840081
:100E30000008F200670884000008083E72020318E8
:100E4000262F700A8400040AF0002B2FF202840A75
:100E5000040AE70000000008F30083136008840020
:100E6000720874020318FF30003C8000F407840A03
:100E7000730843268000840AF30CF30C730C1F39AB
:100E8000203E8000040AE000080047274727641836
:100E9000080083177008840000080F3E0318F92F1C
:100EA0000018E22F083E800A800A840A393E031C9B
:100EB000FB2FE700E71AF42F671A802F67080E3917
:100EC000D83EE70CE7070008D83E031CFB2FF200D2
:100ED000F21BE70AF21BE70A721BE70A3F39E83EFA
:100EE0000318FB2FF20C720C013E4326F300831310
:100EF00067088400000873050319FB2F8006F42F90
:100F0000E43E031CFB2F5F080002031CFB2FF03E96
:100F10000318FB2FEE1FFB2FEE1366030319641457
:100F20008430C900C800CA00C401FB2F8003840AB2
:100F3000383E031CA02FE700F039031DFB2F5E2F66
:100F4000B93E5502403E031CFB2F3039303CF200C5
:100F5000F20E0008F3008313F501530872025408DF
:100F6000031C5607F400F30CF30C730C1F39013EFD
:100F700074020318FB2FE73C0318FB2FF400031443
:100F8000F50C033E031CC02FFE3E0319FB2F720815
:100F9000403E8400750800050319FB2F80066D088C
:100FA0000407D8030339043CF500F50E0310750C53
:100FB000DA074A08031DF42F9E30C900C800043028
:100FC000CA00F42F800B962F800363080319F42FB7
:100FD000840A0002F039031DF42FE3016C08033981
:100FE000C830031D5030D82F8317700884000018B4
:100FF000DB0AF73080008313F00AF00A0800FF3F95
:104200003E007700770077007700770077003E0068
:1042100018001C001E001C001C001C001C001C00C0
:104220003E007700700070003E00070007007F002E
:104230007F0038001C003E007000700077003E00D8
:10424000700078007C007E0077007F0070007000B6
:104250007F00070007003F007000700077003E00FD
:104260003E00770007003F007700770077003E00B0
:104270007F007000700038001C000E000E000E0061
:104280003E00770077003E007700770077003E0021
:104290003E007700770077007E00700077003E00D8
:1042A0003E007700770077007700770077003E00C8
:1042B0001C00220059004D004D00590022001C0036
:1042C0000000B2003D005B00470000000500510007
:1042D0006500290000000200420001004C000000BF
:1042E0000100010038006500500000005B00840000
:1042F0008300200000000B0047003D00000000008C
:02400E00AE3FC3
:084000007F007F007F007F00BC
:00000001FF
